:06000000020033020E9124
:03000B00020E9250
:03001300020EAC2E
:03001B00020EAD25
:03002300020EAE1C
:03002B00020EAF13
:10003300759840758780758921758DFF758BFF7560
:100043008850D299758160758CFA758A0075A8827B
:1000530075900075B0FF7535FF7537FF7539FF75FE
:100063003BFF753DFF753FFF7541FF7543FF7545C9
:10007300FF753600753800753A00753C00753E0013
:1000830075400075420075440075300C753100757C
:100093003404754600754700754800D2A0D2A17894
:1000A3002076FF08B830FAC2A27E80DFFEDEFCC2F3
:1000B30080C287C286D285D284D2A3C2A3DFFEDFE9
:1000C300FEDFFEDFFEDFFED2A3C2A3DFFED2A3C2AA
:1000D300A3DFFEC284D2A3C2A3742812115DDFFE84
:1000E300740812115DDFFE740612115DDFFE7410D9
:1000F30012115DDFFE740C12115DDFFE740112112B
:100103005DDFFEDFFE744012115D7F4090141BE43F
:1001130093121182A3DFF8748012115D7F1490147F
:100123005BE493121182A3DFF874C012115D7F1494
:1001330090146FE493121182A3DFF8DFFEDEFCDF7D
:10014300FEDEFCDFFEDEFCDFFEDEFC748012115DF2
:100153007F14901483E493121182A3DFF874C01206
:10016300115D7F14901497E493121182A3DFF87446
:10017300C012115D74071211827407121182740781
:100183001211827407121182740712118275900082
:10019300D2A0D2A17880E6702575B0FE75A00120AB
:1001A300A00F300019C2007608901317120F988021
:1001B3000D20000AD2007608901319120FB7788128
:1001C300E6702575B0FE75A00220A10F300119C29B
:1001D30001760890131B120F98800D20010AD2019B
:1001E300760890131D120FB77890E6702575B0FB53
:1001F30075A00120A00F301019C210760890131FAC
:10020300120F98800D20100AD21076089013211235
:100213000FB77891E6702575B0FB75A00220A10F8A
:10022300301119C2117608901323120F98800D20F4
:10023300110AD2117608901325120FB77898E67039
:100243002575B0F775A00120A00F301819C21876D4
:1002530008901327120F98800D20180AD2187608D9
:10026300901329120FB77899E6702675B0F775A029
:100273000220A11630191AC2197608E53404B40510
:10028300027402F5341212C88007201904D21976B9
:100293000878A0E6702575B0EF75A00120A00F3097
:1002A3002019C220760890132B120F98800D20205E
:1002B3000AD220760890132D120FB775B0EF75A0F0
:1002C3000220A126753207120EBE120EB0D53206D9
:1002D300753201120EBE120EB775B0EF75A0022073
:1002E300A10820190302123180E378A8E67025756E
:1002F300B0DF75A00120A00F302819C2287608901E
:10030300132F120F98800D20280AD22876089013F5
:1003130031120FB775B0DF75A00220A12675320721
:10032300120EE3120EB0D53206753201120EE3122D
:100333000EB775B0DF75A00220A1082019030212C1
:100343003180E378B0E6702575B0BF75A00120A0B9
:100353000F303019C2307608901333120F98800D86
:1003630020300AD2307608901335120FB775B0BF1C
:1003730075A00220A120753207120F08120EB0D506
:100383003206753201120F08120EB775B0BF75A091
:100393000220A10280E978B8E6702575B07F75A0C8
:1003A3000120A00F303819C2387608901337120F86
:1003B30098800D20380AD2387608901339120FB777
:1003C30075B07F75A00220A120753207120F50125D
:1003D3000EB0D53206753201120F50120EB775B03A
:1003E3007F75A00220A10280E97590FFC2A0C2A17F
:1003F30078C0E6702575B0FE75900120900F3040EF
:1004030019C240760890133B120F98800D20400AC2
:10041300D240760890133D120FB778C1E670257568
:10042300B0FE75900220910F304119C241760890B9
:10043300133F120F98800D20410AD2417608901382
:1004430041120FB778C2E6702575B0FE759004208F
:10045300920F304219C2427608901343120F9880CC
:100463000D20420AD2427608901345120FB778C383
:10047300E6702575B0FE75900820930F304319C2BE
:10048300437608901347120F98800D20430AD243F6
:100493007608901349120FB778C4E6702575B0FE3D
:1004A30075901020940F304419C244760890134B72
:1004B300120F98800D20440AD244760890134D12EF
:1004C3000FB778C5E6702575B0FE75902020950F9F
:1004D300304519C245760890134F120F98800D20AE
:1004E300450AD2457608901351120FB778C6E670C5
:1004F3002575B0FE75904020960F304619C246769A
:1005030008901353120F98800D20460AD24676089E
:10051300901355120FB778C7E6702575B0FE759026
:100523008020970F304719C2477608901357120F50
:1005330098800D20470AD2477608901359120FB7B7
:1005430078D0E6702575B0FB75900120900F305080
:1005530019C250760890135B120F98800D20500A31
:10056300D250760890135D120FB778D1E6702575D7
:10057300B0FB75900220910F305119C2517608904B
:10058300135F120F98800D20510AD25176089013F1
:1005930061120FB778D2E6702575B0FB7590042011
:1005A300920F305219C2527608901363120F98803B
:1005B3000D20520AD2527608901365120FB778D3E2
:1005C300E6702575B0FB75900820930F305319C260
:1005D300537608901367120F98800D20530AD25355
:1005E3007608901369120FB778D4E6702575B0FBBF
:1005F30075901020940F305419C254760890136BE1
:10060300120F98800D20540AD254760890136D125D
:100613000FB778D5E6702575B0FB75902020950F40
:10062300305519C255760890136F120F98800D201C
:10063300550AD2557608901371120FB778D6E67023
:100643002575B0FB75904020960F305619C256762B
:1006530008901373120F98800D20560AD25676080D
:10066300901375120FB778D7E6702575B0FB7590A8
:100673008020970F305719C2577608901377120FBF
:1006830098800D20570AD2577608901379120FB726
:1006930078D8E6702575B0F775900120900F305823
:1006A30019C258760890137B120F98800D20580AB0
:1006B300D258760890137D120FB778D9E670257556
:1006C300B0F775900220910F305919C259760890EE
:1006D300137F120F98800D20590AD2597608901370
:1006E30081120FB778DAE6702575B0F7759004209C
:1006F300920F305A19C25A7608901383120F9880BA
:100703000D205A0AD25A7608901385120FB778DB58
:10071300E6702575B0F775900820930F305B19C20A
:100723005B7608901387120F98800D205B0AD25BCB
:100733007608901389120FB778DCE6702575B0F749
:1007430075901020940F305C19C25C760890138B5F
:10075300120F98800D205C0AD25C760890138D12DC
:100763000FB778DDE6702575B0F775902020950FEB
:10077300305D19C25D760890138F120F98800D209B
:100783005D0AD25D7608901391120FB778DEE6709A
:100793002575B0F775904020960F305E19C25E76CE
:1007A30008901393120F98800D205E0AD25E76088C
:1007B300901395120FB778DFE6702575B0F7759033
:1007C3008020970F305F19C25F7608901397120F3E
:1007D30098800D205F0AD25F7608901399120FB7A5
:1007E30078E0E6702575B0EF75900120900F3060CA
:1007F30019C260760890139B120F98800D20600A2F
:10080300D260760890139D120FB778E1E6702575D4
:10081300B0EF75900220910F306119C26176089094
:10082300139F120F98800D20610AD26176089013EE
:10083300A1120FB778E2E6702575B0EF759004202A
:10084300920F306219C26276089013A3120F988038
:100853000D20620AD26276089013A5120FB778E3CF
:10086300E6702575B0EF75900820930F306319C2B9
:100873006376089013A7120F98800D20630AD26342
:1008830076089013A9120FB778E4E6702575B0EFD8
:1008930075901020940F306419C26476089013ABDE
:1008A300120F98800D20640AD26476089013AD125B
:1008B3000FB778E5E6702575B0EF75902020950F9A
:1008C300306519C26576089013AF120F98800D201A
:1008D300650AD26576089013B1120FB778E6E67011
:1008E3002575B0EF75904020960F306619C2667675
:1008F300089013B3120F98800D20660AD26676080B
:100903009013B5120FB778E7E6702575B0EF7590C1
:100913008020970F306719C26776089013B7120FBC
:1009230098800D20670AD26776089013B9120FB723
:1009330078E8E6702575B0DF75900120900F306878
:1009430019C26876089013BB120F98800D20680AAD
:10095300D26876089013BD120FB778E9E670257553
:10096300B0DF75900220910F306919C26976089043
:1009730013BF120F98800D20690AD269760890136D
:10098300C1120FB778EAE6702575B0DF75900420C1
:10099300920F306A19C26A76089013C3120F9880B7
:1009A3000D206A0AD26A76089013C5120FB778EB46
:1009B300E6702575B0DF75900820930F306B19C270
:1009C3006B76089013C7120F98800D206B0AD26BB9
:1009D30076089013C9120FB778ECE6702575B0DF6F
:1009E30075901020940F306C19C26C76089013CB5D
:1009F300120F98800D206C0AD26C76089013CD12DA
:100A03000FB778EDE6702575B0DF75902020950F50
:100A1300306D19C26D76089013CF120F98800D2098
:100A23006D0AD26D76089013D1120FB778EEE67087
:100A33002575B0DF75904020960F306E19C26E7623
:100A4300089013D3120F98800D206E0AD26E760889
:100A53009013D5120FB778EFE6702575B0DF759058
:100A63008020970F306F19C26F76089013D7120F3B
:100A730098800D206F0AD26F76089013D9120FB7A2
:100A830078F0E6702575B0BF75900120900F307037
:100A930019C27076089013DB120F98800D20700A2C
:100AA300D27076089013DD120FB778F1E6702575D2
:100AB300B0BF75900220910F307119C27176089002
:100AC30013DF120F98800D20710AD27176089013EC
:100AD300E1120FB778F2E6702575B0BF7590042068
:100AE300920F307219C27276089013E3120F988036
:100AF3000D20720AD27276089013E5120FB778F3BD
:100B0300E6702575B0BF75900820930F307319C236
:100B13007376089013E7120F98800D20730AD2732F
:100B230076089013E9120FB778F4E6702575B0BF15
:100B330075901020940F307419C27476089013EBDB
:100B4300120F98800D20740AD27476089013ED1258
:100B53000FB778F5E6702575B0BF75902020950F17
:100B6300307519C27576089013EF120F98800D2017
:100B7300750AD27576089013F1120FB778F6E670FE
:100B83002575B0BF75904020960F307619C27676E2
:100B9300089013F3120F98800D20760AD276760808
:100BA3009013F5120FB778F7E6702575B0BF7590FF
:100BB3008020970F307719C27776089013F7120FBA
:100BC30098800D20770AD27776089013F9120FB721
:100BD30078F8E6702575B07F75900120900F307816
:100BE30019C27876089013FB120F98800D20780AAB
:100BF300D27876089013FD120FB778F9E670257551
:100C0300B07F75900220910F307919C279760890E0
:100C130013FF120F98800D20790AD2797608901469
:100C230001120FB778FAE6702575B07F759004202E
:100C3300920F307A19C27A7608901403120F9880B3
:100C43000D207A0AD27A7608901405120FB778FB32
:100C5300E6702575B07F75900820930F307B19C21D
:100C63007B7608901407120F98800D207B0AD27BA5
:100C73007608901409120FB778FCE6702575B07FDB
:100C830075901020940F307C19C27C760890140B59
:100C9300120F98800D207C0AD27C760890140D12D6
:100CA3000FB778FDE6702575B07F75902020950FFE
:100CB300307D19C27D760890140F120F98800D2095
:100CC3007D0AD27D7608901411120FB778FEE67074
:100CD3002575B07F75904020960F307E19C27E76C1
:100CE30008901413120F98800D207E0AD27E760886
:100CF300901415120FB778FFE6702575B07F7590C5
:100D03008020970F307F19C27F7608901417120F37
:100D130098800D207F0AD27F7608901419120FB79E
:100D23007590FFD2A0D2A17580FFD2A27407B5350A
:100D3300037535FF0535E535A2E092A4A2E192A53E
:100D4300A2E292A6C2AFD2A7C2A7E4B53503020DB1
:100D53008104B53503020DA204B53503020DC304A6
:100D6300B53503020DE404B53503020E0504B535AC
:100D730003020E2604B53503020E47020E68E58012
:100D8300F536A837A936120FD5400624FE500D803C
:100D930005120FDA5006853637120FE1020E89E588
:100DA30080F538A839A938120FD5400624FE500D16
:100DB3008005120FDA5006853839120FF5020E89B5
:100DC300E580F53AA83BA93A120FD5400624FE5018
:100DD3000D8005120FDA5006853A3B121019020EE8
:100DE30089E580F53CA83DA93C120FD5400624FEB9
:100DF300500D8005120FDA5006853C3D12103D025E
:100E03000E89E580F53EA83FA93E120FD540062482
:100E1300FE500D8005120FDA5006853E3F12106119
:100E2300020E89E580F540A841A940120FD540067E
:100E330024FE500D8005120FDA5006854041121032
:100E4300BB020E89E580F542A843A942120FD540A3
:100E53000624FE500D8005120FDA50068542431218
:100E63001115020E89E580F544A845A944120FD552
:100E7300400624FE500D8005120FDA5006854445C6
:100E8300121139020E89D2AF02019002003332C02F
:100E9300D0C0E0C0007880E660011608B800F8759D
:100EA3008CFAD000D0E0D0D032323232327E20DF22
:100EB300FEDEFC227E60DFFEDEFC22748012115D0A
:100EC30005307419B53003753000E5307F04901494
:100ED300ABE530232393121182A3DFF512127F2295
:100EE300748012115D153074FFB53003753018E549
:100EF300307F049014ABE530232393121182A3DFD8
:100F0300F512127F227402B5340D3099FDC2997522
:100F130099C17489020F367403B5340D3099FDC23B
:100F2300997599C2748D020F363099FDC2997599DE
:100F3300C3748512115D3099FDC29905317480B572
:100F43003103753100E531F5991211D3227402B5DD
:100F5300340D3099FDC2997599C17489020F7E745D
:100F630003B5340D3099FDC2997599C2748D020F82
:100F73007E3099FDC2997599C3748512115D3099BC
:100F8300FDC299153174FFB5310375317FE531F534
:100F9300991211D322E4933099FDC299F599A3E4F0
:100FA3009325303099FDC299F599E5333099FDC207
:100FB30099F59922E4933099FDC299F599A3E493A5
:100FC30025303099FDC299F599E43099FDC299F520
:100FD3009922C2D7E89922C2D7E99824FE2274C085
:100FE30012115DE536248030E70264FFF5331212F7
:100FF3001F223099FDC2997599B374C512115D30E2
:1010030099FDC2997599073099FDC299E538C313C3
:10101300F5991211D3223099FDC2997599B174C90A
:1010230012115D3099FDC2997599073099FDC299E6
:10103300E53AC313F5991211D3223099FDC299757C
:1010430099B274CD12115D3099FDC299759907302B
:1010530099FDC299E53CC313F5991211D322309936
:10106300FDC2997599B374C412115D3099FDC2998B
:1010730075995D3099FDC299E53EC313F599309991
:10108300FDC2997599B13099FDC29975995D3099F1
:10109300FDC299E53EC313F5993099FDC29975993F
:1010A300B23099FDC29975995D3099FDC299E53EBB
:1010B300C313F59912121F223099FDC2997599B382
:1010C30074C312115D3099FDC29975995B3099FD16
:1010D300C299E540C313F5993099FDC2997599B149
:1010E3003099FDC29975995B3099FDC299E540C36A
:1010F30013F5993099FDC2997599B23099FDC2994A
:1011030075995B3099FDC299E540C313F5991212A5
:101113001F223099FDC2997599B374C212115D30C3
:1011230099FDC2997599493099FDC299E542C31356
:10113300F59912121F223099FDC2997599B374C1A2
:1011430012115D3099FDC2997599023099FDC299CA
:10115300E544C313F59912121F22C2A2C28033922F
:1011630087339286339285339284D2A3C2A3339278
:1011730087339286339285339284D2A3C2A322C249
:10118300A2D280339287339286339285339284D26C
:10119300A3C2A3339287339286339285339284D248
:1011A300A3C2A32275F064842430121182740AC589
:1011B300F0842430121182E5F0243012118222755A
:1011C300F00A842430121182C5F0243012118222D5
:1011D300D2D575F064847004C2D574F02430121132
:1011E30082740AC5F084700520D50274F02430128D
:1011F3001182E5F024301211822275F00A84700204
:1012030074F02430121182E5F0243012118222E4AA
:1012130093A3B45E0122121182021212700474208D
:101223008008C313C313C313C313121182221212F0
:101233007F3099FDC2997599B13099FDC29975991D
:10124300783099FDC2997599003099FDC2997599C5
:10125300B23099FDC2997599783099FDC299759903
:10126300003099FDC2997599B33099FDC29975996A
:10127300783099FDC2997599000200333099FDC207
:10128300997599B13099FDC29975997B3099FDC2D1
:10129300997599003099FDC2997599B23099FDC23B
:1012A3009975997B3099FDC2997599003099FDC262
:1012B300997599B33099FDC29975997B3099FDC29F
:1012C3009975990022748412115D7420121182742D
:1012D3008812115D7420121182748C12115D7420B6
:1012E3001211827402B5340B8531488546317488F6
:1012F30002130E7403B5340B853146854731748C64
:1013030002130E853147854831748412115D747E52
:1013130012118222922280229223802392248224F9
:101323009225822592268226922782279228822836
:1013330092298229922A822A93298329932A832A0A
:10134300932B832B932C832C932D832D932E832EDE
:10135300932F832F933083309331833193328332AE
:10136300933383339334833493358335933683367E
:10137300933783379338833893398339933A833A4E
:10138300933B833B933C833C933D833D933E833E1E
:10139300933F833F934083409341834193428342EE
:1013A30093438343934483449345834593468346BE
:1013B300934783479348834893498349934A834A8E
:1013C300934B834B934C834C934D834D934E834E5E
:1013D300934F834F9350835093518351911F811F98
:1013E30091208120912181219122812291238123A6
:1013F3009124812491258125912681269127812776
:101403009128812891298129912A812A921F821F5B
:10141300922082209221822100000000000000100F
:101423000000000000001018000000000010181C4D
:101433000000000010181C1E00000010181C1E1FC6
:10144300000010181C1E1F1F0010181C1E1F1F1F3A
:1014530010181C1E1F1F1F1F4D757A796B616E7448
:101463002036202076312E302020202020736D69F5
:10147300616C656B2E7072762E706C20202020209C
:10148300204320207E2020302020203020202030A8
:1014930020202020202020202031323720313237D5
:1014A30020313237202020202D4320202D44657306
:1014B3002D4420202D4573202D4520202D4620200E
:1014C3002D4765732D4720202D4173202D4120206A
:1014D3002D4220202D482020204320202B436973B8
:1014E3002B4420202B4469732B4520202B4620209E
:1014F3002B4669732B4720202B4769732B412020F0
:101503002B4169732B4820202B432020204D757AD3
:10151300796B616E7420362076312E302032303074
:10152300372D30362D3239202863294164616D20EF
:10153300536D69616C656B206A616E6B6F6D757A53
:10154300796B616E744077702E706C207777772E8D
:10155300736D69616C656B2E7072762E706C20579B
:10156300737A656C6B6965207072617761207A614B
:101573007374727A657A6F6E652E204A616B696542
:101583006B6F6C7769656B207A6173746F736F77B8
:10159300616E6961206B6F6D657263796A6E652038
:1015A3006B6F6475206E6965646F7A776F6C6F6EAD
:1015B300652E20416C6C20526967687473205265F4
:1015C3007365727665642E204672656520666F7258
:1015D300206E6F6E20636F6D6D65726369616C2041
:0615E3006F6E6C792E20F2
:00000001FF
